:020000040000FA
:10000000830100308A000428203084002630162026
:1000100083010730AA00FD30A90026308400293072
:100020001A2083010D2F04068001840A0406031D93
:1000300013280034F00025208000840A040870068C
:10004000031900341B288312A900AA1B2E282A0892
:100050008A002908A90A0319AA0A820083132A1808
:0C00600083172908A90A84000008080082
:100E1A000330831285000730990083169F0123301F
:100E2A0085008C018B010530831292000B138B1302
:100E3A000C30950093018C1C902F64008C102508AF
:100E4A002404230422040319712F0130F000F10154
:100E5A00F201F301A2027108031C710FA3027208C6
:100E6A00031C720FA4027308031C730AA502003044
:100E7A002502031D4A2F00302402031D4A2F1E306B
:100E8A002302031D4A2FE1302202031C512FFF3097
:100E9A009300303095047F2F00302502031D5F2F09
:100EAA0000302402031D5F2F00302302031D5F2F31
:100EBA0065302202031C6D2F130803197F2FA10826
:100ECA000319692FA1037F2F93031E30A1007F2FDF
:100EDA00CF30950593017F2F2330831696000B1090
:100EEA008B1563008B1196015A308312A200A3015D
:100EFA00A401A50105082339033AA000A60803198D
:100F0A00902F2008270603198F2F2008A7000830E2
:100F1A00A600902FA603A608031D202F280827063F
:100F2A00F000701CBF2F271CA12F4030A200773081
:100F3A00A3001B30A400BE2FA718BF2FA71EA92FDE
:100F4A00E030A2001E30BC2F00302502031DB72F4F
:100F5A0000302402031DB72F1E302302031DB72FB2
:100F6A00E1302202031CBF2FD030A2007430A3004C
:100F7A00A401A50127082806F000F01CD42FA71CFD
:100F8A00CD2F4030A2007730A3001B30A400D32F0E
:100F9A002718D42F6430A200A301A401A5012808B0
:100FAA002706F000F01EF82F271CA718F82FA71EF7
:100FBA00F22F00302502031DEC2F00302402031DFE
:100FCA00EC2F1E302302031DEC2FE1302202031CFA
:100FDA00F82FE030A2001E30F52FD030A200743076
:100FEA00A300A401A5010830A6002708A800202F05
:060FFA0008340334033447
:02400E00E4329A
:00000001FF
